:1000000010C02AC029C028C027C026C025C024C0CF
:1000100023C022C021C020C01FC01EC01DC01CC0E4
:100020001BC011241FBECFE5D2E0DEBFCDBF10E064
:10003000A0E6B0E0E0E4F4E002C005900D92A23644
:10004000B107D9F710E0A2E6B0E001C01D92A736D3
:10005000B107E1F78ED0F2C1D3CF81E88ABB8FE13F
:1000600087BB089590916000981789F098B3987FA6
:1000700098BBDF9828B3982F9770922B98BB2BB31F
:10008000982F92959078922B9BBB80936000089557
:100090001F93CF93DF93EC011091600080E0E2DFCB
:1000A00020E030E003C000002F5F3F4F2C173D07DA
:1000B000D4F3812FD7DFDF91CF911F91089585E091
:1000C000D1DF8FE39DE0A3E081509040A040E1F7B5
:1000D00000C0000080E0C6DFA7EAB1E61197F1F7A3
:1000E00000C000008AE0BEDF8FE39DE0A3E0815006
:1000F0009040A040E1F700C0000080E0B3DF089529
:100100000F931F93D89800C000C00000D89A23E036
:100110002A95F1F70000D89880E090E001C0000037
:10012000C9990CC0019621E6893A9207C1F706C029
:100130006F5F7F4F8F4F9F4F000003C060E070E004
:10014000CB01C99B08C0603523EC720720E0820711
:1001500020E0920769F7665F7F4F8F4F9F4F2AE03D
:1001600030E040E050E019D1B901CA011F910F9170
:100170000895BF92CF92DF92EF92FF920F931F9359
:10018000CF93DF9383E294EF0197F1F700C0000073
:1001900064DFA1EEB4E01197F1F700C0000080E049
:1001A00061DFCD9913C02FE936E841E0215030409E
:1001B0004040E1F700C0000082DF8FE996E8A1E04F
:1001C00081509040A040E1F700C00000A3ECB9E0EE
:1001D0001197F1F700C00000D69A83EC99E00197DF
:1001E000F1F700C000008BB390E489278BBB2FE9A7
:1001F00036E841E0215030404040E1F700C00000C7
:100200008BB389278BBB8FE996E8A1E081509040A2
:10021000A040E1F700C00000C0E0D0E000E010E046
:10022000BB24B39422E3E22EF12C95E0C92E80E4A6
:10023000D82E0F5F1F4F64DF6A30710514F4DE9A09
:1002400001C0DE9880916400813009F082C0CD99B0
:1002500017C090916600992319F48093660002C03C
:10026000109266008BB38D258BBB2FE33DE043E0FE
:10027000215030404040E1F700C0000003E010E0B2
:100280006A307105C4F42196C932D10514F486E0B0
:1002900004C0C13AD10514F489E0E4DE8091600025
:1002A0008093650087EE93E00197F1F700C00000AE
:1002B00080E0D8DE5CC0C801B7015CD0009709F1CE
:1002C00081309105D9F480916500853059F5809190
:1002D0006600813039F580E0C5DE89E0C3DEA7EB3A
:1002E000B8E81197F1F700C0000080E0BBDE8FE0B6
:1002F00097E20197F1F700C000009BCF8230910593
:1003000089F480916500853069F4809166008130C0
:1003100049F480E0A7DE86E0A5DEA7E9BAE31197FD
:10032000F1F7E1CF80916500863011F0893011F44A
:10033000209709F485E096DEC0926500AFECB7E047
:100340001197F1F700C0000080E08CDEC0E0D0E043
:1003500070CFCD996ECFB0926400DE982FE33DE070
:1003600043E0215030404040E1F700C0000003E08E
:1003700010E05FCF97FB092E07260AD077FD04D047
:1003800027D006D000201AF4709561957F4F08950C
:10039000F6F7909581959F4F089597FB092E0526B6
:1003A0000ED057FD04D028D00AD0001C38F4509548
:1003B0004095309521953F4F4F4F5F4F0895F6F789
:1003C00090958095709561957F4F8F4F9F4F0895C1
:1003D000AA1BBB1B51E107C0AA1FBB1FA617B7076B
:1003E00010F0A61BB70B881F991F5A95A9F7809587
:1003F0009095BC01CD010895A1E21A2EAA1BBB1B4A
:10040000FD010DC0AA1FBB1FEE1FFF1FA217B307E0
:10041000E407F50720F0A21BB30BE40BF50B661FF6
:10042000771F881F991F1A9469F7609570958095BA
:1004300090959B01AC01BD01CF010895F894FFCFC9
:02044000FF00BB
:00000001FF
